:10000000112484B714BE81FF18D185E08EBD8EE027
:1000100000D1D49AD29A86E023EC3FEF91E03DBD27
:100020002CBD9BB9589BFECFCC9AA8958150B9F7AF
:10003000BB24B39425E0A22E9FE7D92E8EECC82EC8
:10004000D4D0813421F481E0F0D083E0B5C0823493
:1000500011F484E103C0853419F485E0E6D0B3C01F
:10006000853569F4C2D0E82EFF24BFD0082F10E0F8
:10007000102F00270E291F29000F111FA3C086353E
:1000800021F484E0D2D080E097C0843609F060C0CB
:10009000ACD0ABD0F82EA9D0C0E0D1E0A6D08993E7
:1000A000FC16E1F783E0F80187BFE895B6D007B604
:1000B00000FCFDCF0115110511F0A8012AC08091A7
:1000C00000012091010130E0322F222790E0282BFF
:1000D000392B309385012093840140910801809150
:1000E000090190E0982F882750E0842B952B90935E
:1000F0008701809386012450304020930801232FEC
:10010000332720930901D0920001C092010140E001
:1001100050E0A0E0B1E02C9130E011968C91119765
:1001200090E0982F8827822B932B1296FA010C01CE
:10013000B7BEE89511244E5F5F4FF1E0A034BF07D2
:1001400051F7F801A7BEE89507B600FCFDCF3BC00C
:10015000843751F54AD049D0F82E47D05ED0E80117
:10016000EF2C209719F48091840114C0C130D1057F
:1001700019F4809185010EC0C830D10519F4809121
:10018000860108C0C930D10519F48091870102C0E9
:10019000FE01849121961AD0EA9419F70F5F1F4F40
:1001A000FA940F0D111D0FC0853741F436D08EE142
:1001B0000DD083E90BD08CE009D005C0813511F456
:1001C00088E027D02AD080E101D03ACF2AE030E081
:1001D0008095089410F4DA9802C0DA9A000015D0DD
:1001E00014D086952A95B1F70895A89529E030E0B6
:1001F000CB99FECF0AD009D008D08894CB99089427
:100200002A9511F08795F7CF08959EE09A95F1F71A
:10021000089598E191BD81BD0895E7DF803219F01E
:1002200088E0F7DFFFCF84E1D1CF1F93182FDDDF08
:100230001150E9F7F2DF1F91089580E0EADFE4E072
:04024000FF270994F7
:021EFE000104DD
:00000001FF
